:020000040000FA
:1000000083128501860183162D30850086016030BC
:100010008F008F309F00831241309F00A001A1010B
:10002000A201A3010A30A500051320082C20860098
:1000300005167E20051221082C20860085177E20BB
:10004000851322082C20860005177E20A503031D9A
:1000500014283A20592012280F398207E7344434F3
:10006000AE346E344D346B34EB344634EF346F348D
:100070000834A3341F151F193B2883161E0883124A
:10008000A3001E08A4000800FF30A000A1006430F7
:10009000A00AA3020301031C013EA402031847287F
:1000A00064302307F63EA10A031852280A3EA20034
:1000B00008006030A3020130031C013EA4020318B3
:1000C00065280A30A000A1000800230803178D004E
:1000D00083168C130C1483120C080313A000A100C8
:1000E000A300A00E0F30A005A1050B30A200253003
:1000F000230203188514031C851008000630A6008F
:0E010000FA30FF3E031D8128A60B8028080060
:02400E00103F61
:10420000F034F034F034F134F134F134F134F13489
:10421000F234F234F234F234F234F334F334F3346B
:10422000F334F334F434F434F434F434F434F5344F
:10423000F534F534F534F534F534F634F634F63433
:10424000F634F634F734F734F734F734F734F83417
:10425000F834F834F834F834F934F934F934F934FA
:10426000F934103410341034103410341134113443
:104270001134113411341134123412341234123412
:1042800012341334133413341334133414341434F5
:1042900014341434143415341534153415341534D9
:1042A00016341634163416341634163417341734BC
:1042B00017341734173418341834183418341834A1
:1042C0001934193419341934193420342034203471
:1042D0002034203421342134213421342134223437
:1042E000223422342234223422342334233423341B
:1042F00023342334243424342434243424342534FF
:1043000025342534253425342634263426342634E1
:1043100026342734273427342734273427342834C5
:1043200028342834283428342934293429342934A9
:104330002934303430343034303430343134313462
:104340003134313431343234323432343234323440
:104350003334333433343334333433343434343423
:104360003434343434343534353435343534353408
:1043700036343634363436343634373437343734EA
:1043800037343734383438343834383438343834CF
:1043900039343934393439343934403440344034A0
:1043A0004034403441344134413441344134423466
:1043B0004234423442344234433443344334433449
:1043C000433444344434443444344434443445342D
:1043D0004534453445344534463446344634463411
:1043E00046344734473447344734473448344834F4
:1043F00048344834483449344934493449344934D8
:00000001FF
